:020000040000FA
:10000000642B00340034FF3FCF000308CE00B30858
:100010000319B203B30B1928B208031D19280F30B6
:10002000B2003508B3003608B4070318B30A3B1C06
:100030003B170B114E088300CF0E4F0E09003008FE
:10004000B1000A30BA00B10B34282608B800C2212A
:100050003908A1003708A2002708B800C2213908D2
:10006000A3003708A4000800B10B5C282808B800DA
:10007000C2213908A1003708A2002908B800C2210E
:100080003908A3003708A400430B080029080F3ED5
:10009000A30029081B3EA40008003F08B800C221A5
:1000A00008003B122830A3003708A20008003908D6
:1000B000A2003708A3000800B10B7B280C30A40075
:1000C000BF1F71283B162930A100BF09BF0A4D2070
:1000D0003908003C031951203B1A57200330B00067
:1000E0007A283F08B800C2213908A1003708A200C9
:1000F0002830A3000800B10B90282630C500183026
:10010000C600FF30C70076212A30A1001930A200B6
:100110002608B800C2213908A3003708A400080047
:10012000B10BA5282730C5003C30C600FF30C70002
:1001300076212B30A1002B30A2002708B800C22165
:100140003908A3003708A4000800B10BC6282930DD
:10015000C5000D30C6000030C7007621BB1DB22897
:10016000B52295212C30A1002B30A2002908B8001F
:10017000C2213908A3003708A400430B080029084E
:100180000F3EA30029081B3EA4000800B10BDB288A
:100190002830C5002B08C6000030C70076212C305F
:1001A000A1002C30A2002808B800C2213908A30001
:1001B0003708A4000800B10BF6282A30C5006430C7
:1001C000C600FF30C7007621BB1DEA28B522952165
:1001D0000A30BA002C30A1002D30A2002A08B80045
:1001E000C2213908A3003708A4000800B10B0B296D
:1001F0004330C5000330C6000030C70076212C30E4
:10020000A1002E30A2004308B800C2213908A30083
:100210003708A4000800B10B20294030C5003C304D
:10022000C6000130C70076212E30A1002E30A2007A
:100230004008B800C2213908A3003708A40008000C
:10024000B10B35294130C5003C30C600FF30C70036
:1002500076212E30A1002C30A2004108B800C22126
:100260003908A3003708A4000800B10B4A2942301E
:10027000C5003C30C600FF30C70076212E30A100FB
:100280001D30A2004208B800C2213908A300370877
:10029000A4000800B10B61293530C5000030C6004C
:1002A000FF30C70076211830A1002A30A20010309C
:1002B000BA003508B800C2213908A3003708A400E5
:1002C00008003630C5000030C600FF30C700762178
:1002D0001830A1002F30A2001030BA003608B80044
:1002E000C2213908A3003708A4000800BB187B29E5
:1002F0003B198829080045088400800A0008460246
:10030000031D08004508840047088000800A080093
:1003100045088400800300084702031D08004508C3
:10032000840046088000800308002B08B700B7034C
:100330003708280203190800B70B98299F292B08B2
:10034000B700B7033708A8000800831603139B0003
:10035000831603131C14831603131A088312031342
:100360000800831603131C158B138B1BB4295530FF
:100370009D00AA309D009C14831203139C131C1132
:100380008B170800B701B9010830A500B80DB70DEB
:100390003A0837020318B700B90DA50BC6290800A3
:1003A0000030850083160313061786150615831281
:1003B00003130301013E7A22061FF2211C2213229D
:1003C0008316031306138611061183120313080004
:1003D000362B08003F2B08003B100130B0004008CE
:1003E000AD000800AF08031D08003B18FB290330CF
:1003F000B000A0013B14B00A3030AF0030080F3C11
:10040000031D052AEC218E23A1231F20742208003E
:10041000AF08031D08003B1C08000619102A1D2AFE
:1004200086190800142A082ABB14BB153030AF0007
:100430001F20BB10BB110800082A3B15BB1530302C
:10044000AF001F203B11BB1108002C0882070034AD
:100450000234043408343034C4012C08023C03193B
:10046000352AAE194414352A2C2A00308500203054
:100470002C0784000008A521441C2E068600452A6E
:100480000430AC0002308A00342A25228500043072
:10049000A500FF307A22A50B492AAF080319512A7B
:1004A000AF03AC0B442A08003B13A00A20083C3CD5
:1004B00003198122AD0B722AB00A3008043C0319DB
:1004C000EC213003403E84000008AD00AD08031964
:1004D0005C2A3008013C0319E8213008033C031969
:1004E000EA211F207422CD2B300B782A7E22792A14
:1004F000AE010800FF3E031D7A2A08000830AE0650
:100500000800A001A70A27083C3C031990222608EE
:10051000183C0319932229080D3C03199E221F2819
:10052000A701A60A0800A601A80A2B082802031D95
:1005300008000130A800A90AB52208000130A9006E
:10054000AA0AB52208001D30AB000430BA002A0800
:10055000B800C2213708003C0319B22208001F303E
:10056000AB0008001E30AB0008002030AB002908AB
:10057000043C0319AF222908063C0319AF222908BD
:10058000093C0319AF2229080B3C0319AF222908A3
:10059000023C0319A32208008316051483120800E5
:1005A0008316051083120800D02205100301AB3E0C
:1005B0007A22CC220301033E7A220800A50103011E
:1005C000103E7A22051C251405180800E42A811F14
:1005D0000800011F0800811E0800811F0800ED2A85
:1005E000E722D022051000000000000000000000FB
:1005F000CC2203010F3E7A220F2BD02205100301DB
:100600000E3E7A22CC220000000000000000000014
:1006100000000F2B0830A5003D1CFD2AF02ABD0C60
:10062000031CBD13A50B0C2B08000830A500E72206
:1006300083160510831205100000000000008316C9
:10064000051483120000000000000000051C2A2B86
:10065000BD172B2BBD1303010F3E7A22250B312B27
:100660000800BD0C031CBD13A503172BD422DE22EA
:10067000CC30BD000A234430BD000A23E929BF0164
:10068000D422DE22251CEB29CC30BD000A23BE304B
:10069000BD000A2315233D08BE0015233D08BF00F9
:1006A000D422BE0CBE0CBE0CBE0C3E16BE163E17AF
:1006B0003F1C3E12BF1CBE123F1D3E13BE173F1E05
:1006C000BE133E08BF00EB29883083160313810058
:1006D0008312031307309F008501860183160313DD
:1006E000860101308500831203138030BB00A00116
:1006F000AE013030AF008E239523B5224008AD0007
:100700000130B0001F20E821A0308B000F30B20074
:100710003508B300B30A3608B400CB2B0B30A50064
:100720003A30C80003308A0008004808A521C500F7
:100730002508BA23840045088000C803A50B952B23
:1007400008002508BA23C7234808831603139B0013
:10075000831203134508831603139A00B1211F3037
:10076000BC000301FF3E7A22BC0BB12BC803A50BD2
:10077000A12B08008207003426342734283429347A
:100780002A344334403441344234353436348400DE
:100790000008C50008003B1B542AD0214022CB2B67
:1007A000FF3FFF3FFF3FFF3FFF3FFF3FFF3FFF3F59
:1007B000FF3FFF3FFF3FFF3FFF3FFF3FFF3FFF3F49
:1007C000FF3FFF3FFF3FFF3FFF3FFF3FFF3FFF3F39
:1007D000FF3FFF3FFF3FFF3FFF3FFF3FFF3FFF3F29
:10420000E700240057003700B400B300F300260095
:10421000F700B700F600F100C3007500D300D2002C
:104220006700D200E600F600E60067006700F600CF
:10423000B300710070007500F600D300F600D600E0
:10424000B500E500C100E500D30051007100D300C6
:1042500096001000F00070007500B500D100C0009D
:104260000E002E00190002000B00010008000200E1
:10427000030042004000FF00FF00FF00FF00FF00BE
:10428000FF00FF00FF00FF00FF00FF00FF00FF0036
:10429000FF00FF00FF00FF00FF00FF00FF00FF0026
:1042A000FF00FF00FF00FF00FF00FF00FF00FF0016
:1042B000FF00FF00FF00FF00FF00FF00FF00FF0006
:1042C000FF00FF00FF00FF00FF00FF00FF00FF00F6
:1042D000FF00FF00FF00FF00FF00FF00FF00FF00E6
:1042E000FF00FF00FF00FF00FF00FF00FF00FF00D6
:1042F000FF00FF00FF00FF00FF00FF00FF00FF00C6
:02400E00213F50
:08400000FF3FFF3FFF3FFF3FC0
:00000001FF
